:030000000219FDE5
:03000B000200AA46
:03002B0002015C73
:03005B000202F9A5
:030073000202E6A0
:1000800002030406080C10182030406080040608A3
:100090000C10182030406080A0C00003070F1F0D17
:1000A0000D04050D050305030302C2AFC0D0C0E077
:1000B000206214E5256009E473E525F4F58AD2622F
:1000C000D0E0D0D0D2AF3285268AC262E526F46075
:1000D0002F30682520720DD0E0D0D0C292C291C2DC
:1000E00090D2AF32C292C291C290206F0C206609AA
:1000F0007405D5E0FDE57B4290D0E0D0D0D2AF32A0
:10010000758A00C28DD26201F901B9306805206696
:1001100002D29201B9306805206602D29101B9304D
:100120006805206602D29001B9C29530680A20663F
:1001300007740CD5E0FDD29201B9C29430680A2050
:100140006607740CD5E0FDD29101B9C29330680AFC
:10015000206607740CD5E0FDD29001B9C2AFC2ADE4
:1001600053E6EFC0D0C0E0D2D3D2AFC2CEE52A6012
:1001700007207449152A21BD7800790020742EE5E6
:1001800080307E01F430E70278FF53DACF207E031F
:1001900043DA20307E0343DA10C2D8C271E58030E2
:1001A0007E01F430E70279FFC3E89970CB30610338
:1001B000752A18207403752A18885CD27020740D73
:1001C000E52B6004152B21CD43DA01C2D820700243
:1001D000413CA85C206102C2702074367982B70469
:1001E00031C3E894F0400374F0F8E8C4540F28F8E1
:1001F0007984B703024112C313C313872120080275
:10020000C313200A06C3C898F8411228F850037493
:10021000FFF88822E52D54066022206B1FE536C3C7
:1002200033C333F8E564C313C313F9C39522400203
:100230008922E82522F52250037522FF7882B60430
:1002400059852224A824C3E52495614002A861C3EE
:10025000E895634002A8638825E5667002418DC376
:10026000E8AA669A5003E8FAE4F9EAC333FBE568C2
:10027000F45B29400D2567F8E56760021567400BC0
:10028000418D0AC3E5679A5002056778FF8826C248
:100290006FC3E52694F84002D26FC3E52594404031
:1002A00002D26420CF0AD0E0D0D043E610D2AD32E3
:1002B000C2CF053A7801E52A6005307402152AC3D9
:1002C000E55C94014005755F0041DC75600075696F
:1002D00000E55F2401F55F5003755FFFD0E0D0D0EB
:1002E00043E610D2AD32C2AF53E67F7592FA7593F2
:1002F000FFC260759104D2AF32C2AF53E6EFC2AD18
:10030000C0D0C0E0C0F0D2D3D2AFA8FBA9FCC2D805
:10031000307102616053DACF207E0343DA10307E01
:100320000343DA20D271E580307E01F420E70261D8
:100330003788278928A18D53DACF207E0343DA201E
:10034000307E0343DA10C2D8C271307402A17978CA
:1003500000E580307E01F430E702A179885CA1617C
:1003600053DACF207E0343DA20307E0343DA10C213
:1003700071206102813953DACF207E0343DA1030D5
:100380007E0343DA20C2D8D27188578958C3E895D2
:1003900055F8E99556F97B007E087A00C3E8948CFD
:1003A000E994005005755B00812B882178A2E6A8AE
:1003B000216055C3E894C8E994005008E4D2E4FBF6
:1003C0007A0A8106C3E89468E994015008E4D2E30C
:1003D000FB7A0F8106C3E894D0E994025008E4D276
:1003E000E2FB7A1E8106C3E894A0E994055008E474
:1003F000D2E1FB7A3C8106C3E89498E9940850085E
:10040000E4D2E0FB7A787E00C3E89559FCE9955A7E
:10041000FD30E70AECF42401FCEDF43400FD755BDB
:1004200000C3EC9AED9E5003755B018859895A858B
:1004300057558558567802A161C3E89527F8E99584
:1004400028F9307C02A145307B02A145307A02A117
:100450003E207502815CE9FDE8FC817BE9C313F96C
:10046000E813F8307902A13EE9C313F9E813F83034
:0F0470007802A13EE9C313FDE813FC20612CC301
:10047F00EC941CED940240028192ED701EC3EC943B
:10048F00C850180529E52970021529C3E529940AD2
:10049F005002A179755C00D270A179E5296002152F
:1004AF00297888E6F97400207F087896B9030278D6
:1004BF009EE624FAFEE43400FFC3EC9EFCED9FFDA4
:1004CF009208B90310A2085007207609D27681E46A
:1004DF00307602C276A2085016B9030DECF424014F
:1004EF00FCEDF43400FD0204FE78007900A145B95B
:1004FF000315EC33FCED33FDC3EC940AFCED9400D3
:10050F00FD50047C007D00C3EC94FFED9400400689
:10051F0078FF7900A145EC8572F0A4C5F0A2F733FE
:10052F00F87900400302056178FF7900020561E95F
:10053F00C313F9E813F8307C0EE9600278FFC3E8C3
:10054F001338F8E43400F9C3E894FFE9940040024B
:10055F0078FF885CD270206102A179741FF4552F47
:10056F004BF52FC274EB7002D274752A18307403D6
:10057F00752A0A306102A18D20740353DAFE2074AC
:10058F0003752B06D0F0D0E0D0D0D2AD43E61032B9
:10059F0079010205BD79030205BD790A0205BD790E
:1005AF001E0205BD79640205BD79C80205BD781725
:1005BF00E4D5E0FDD8FAD9F6227A147B780205E467
:1005CF007A107B8C0205E47A0D7BB40205E47A0B7A
:1005DF007BC80205E47902E4C294D5E0FDD291D53F
:1005EF00E0FDC291D5E0FDD294D5E0FDE920E00217
:1005FF00D29230E002D290E573D5E0FDE920E0021F
:10060F00C29230E002C2907496D5E0FDD9C9EAF8E3
:10061F00D5E0FDD8FBDBBEC29422C37C007D007504
:10062F00F00005F0EA33FAEB33FB50F6EB13FBEA7D
:10063F0013FAC3E9FFE8FEE89AF8E99BF95004EFD3
:10064F00F9EEF8B3EC33FCED33FDD5F0DFEDF9EC5B
:10065F00F822E889F08A20D2D4F8A9F07B0030F78D
:10066F000B7BFFF42401F8E9F43400F9E88520F05E
:10067F00A4ADF0F8E98520F0A4AFF0FEED2EF974EB
:10068F00003FFA7C04C3EA13FAE913F9E813F8DC24
:10069F00F48BF030F70AE8F42401F8E9F43400F9A8
:1006AF00E889F0C2D4F8A9F0227882B604030207D1
:1006BF0013C3E55C940140030206DD852224E4F5B3
:1006CF0044F545F546F547F548C26E0207137882A3
:1006DF00E6FCD26EE522F523783879C7AA40AB4104
:1006EF00C3EB13FBEA13FAEC146013C3EB13FBEA2F
:1006FF0013FAEC14146007C3EB13FBEA13FAD129B6
:10070F008844894522C3E5449523F8E5459400F9CB
:10071F00500CC3E89480E994FF4016020744C3E8E5
:10072F00947FE994005003020744787F7900020711
:10073F0044788079FF8849894A22E5492546F8E5BA
:10074F004A3547F9854A20E4300701F43548FA3035
:10075F00E709C3EA94F04015020782C3EA940F50E9
:10076F000302078278FF79FF7A0F020782780079F8
:10077F00007AF0C3E5249561500AC37401952450A3
:10078F000B0207A0E54A20E70E0207A0E54A30E773
:10079F0006884689478A482278A5E6FAC3E5493391
:1007AF00F8E54A33F9D161E930E70BC3E89480E902
:1007BF0094FF4013E1DAC3E8947FE994005002E11B
:1007CF00DA787F7900E1DA788079FFE820E715C3DE
:1007DF00E52398F84009C3E8940140030208017823
:1007EF0001020801E8F424012523F840030208015F
:1007FF0078FF884B2278A6E6FAA847A94812066127
:10080F00E930E70CC3E89401E994FF40160208367B
:10081F00C3E894FFE99400500302083678FF79008B
:10082F00020836780179FFE920E715C3E54B98F800
:10083F004009C3E89401400302085D780102085D96
:10084F00E8F42401254BF8400302085D78FF882463
:10085F002278FFC26420693D206A12D264C3E54149
:0F086F00940A4009C3E52594405002C26479A160
:10087E00E76023E541601F74FF8541F0848539F000
:10088E00306A0375F005A4F8C5F0600278FFC3E87E
:10089E0095645002A864886322C3E5409440E54104
:1008AE009401E56350031401B8046002F56322025B
:1008BE0008C02275E890227883E6FFE5E820ECF781
:1008CE00A8BDA9BE0570C3E57094084052757000AE
:1008DE00E9FA79A0E76044EA7007E571601B020847
:1008EE00FBC3E895716010E5715006600C140209A7
:1008FE00070460F9020907E571F571C3946D401B99
:10090E007561C0C394044013756180C39404400B99
:10091E00756140C39404400375610075BB0622E502
:10092E00612410500274FFF5617982B704022154DC
:10093E00C3A861E524985002A824C3E89563400239
:10094E00A86388258826E570B4070375BB1022744A
:10095E003279A787F0A4C5F0A2F733F8C3E8956102
:10096E004002A861882288248825882688642275FA
:10097E0040007541F022C2AF75C820A8CCA9CDAAFF
:10098E003A30CF010A75C824D2AFAB3BAC3C883BA2
:10099E00893CC3E89BF8E99C206908F9306702415D
:1009AE009021EDAD3D8A3DF9EA9DFA600478FF791C
:1009BE00FFAE3EAF3F8B3E8C3FA83BA93CC3E89EAB
:1009CE00F8E99FF9C3E54113FBE54013FAE82AF570
:1009DE0040E93BF54150067540FF7541FF4137AA8E
:1009EE0040AB41AC40AD417E047F02C3EB9404406A
:1009FE00021E1FC3EB940840021E1FC3ED13FDEC35
:100A0E0013FCDEF7C3EA9CFAEB9DFBEF6009C3E92A
:100A1E0013F9E813F8DFF7EA28FAEB39FB8A408B73
:100A2E004150067BFF8B408B41C3EB94025002D2A8
:100A3E00673069047F0341627892E6FFC3E537941D
:100A4E008240110FC3E53794A040010FC3EF940607
:100A5E0040027F057E02E541C4540FF9E541C454BE
:100A6E00F0F8E540C4540F28F8C3E89EFAE9940064
:100A7E00FB4009C3EA9402EB940050047A02E4FBB3
:100A8E0041DCAA40AB41EBC4FEEAC4540F4EFCC39A
:100A9E00EA9CFAEB9400FBC3E813C313F8EA28FAB6
:100AAE00EB3400FB8A408B41C3EB94024002C267D9
:100ABE007802EBC4FE7B00EAC4540F4EFAC3EA98E8
:100ACE00FA4005C3940250027A027892E6FF306033
:100ADE000241DC855192855293D26043E680C3E495
:100AEE009AF8E49BF93067026168E8FAE9FBD3E90A
:100AFE0013FDE813FC88518952C3EF94036038EF5D
:100B0E0020E00DE82CF8E93DF9ECFAEDFB020B3193
:100B1E00E828F8E939F9C3E82402F8E93400F97A4B
:100B2E00FE7BFFC3EF9403400E8A538B54884D898E
:100B3E004E8C4F8D50619C885389548A4D8B4E8CB0
:100B4E004F8D503069127553F07554FF754FF07517
:100B5E0050FF7551F07552FF619CE8FAD3E813FC13
:100B6E008851C3EF94036020EF20E007E82CF8ECE7
:100B7E00FA6188E8282402F87AFEC3EF940340084D
:100B8E008A53884D8C4F619C88538A4D8C4FE568F3
:100B9E00C3335002646BF56830600261A67534028F
:100BAE00D26043E680E52D54066034A840A941C3C7
:100BBE00E913F9E813F8C3E913F9E813F8306904F7
:100BCE00E92440F9C2AF53E67F759100C3E498F56E
:100BDE0094E499F595759104D26043E680D2AF22E4
:100BEE00D265754300752000306C03752040020CF1
:100BFE000DD265754300752040306C03752000786A
:100C0E00017901206720E52D54066002C265791432
:100C1E00E541C313700104F8C394144002781430F4
:100C2E006904781B791B206010E543600C30690362
:100C3E00D53404D26D81B071AE0543E59BF45440BA
:100C4E00B52002819A30690908C3E89940011881DC
:100C5E003420650A08C3E8994002810D8134C265CB
:0E0C6E00C2AF53E67F75910030671275940097
:100C7C007595FE759104D26043E680D2AF810DAEBE
:100C8C0040AF41C3E49EF594E49FF595817FC3E5A5
:100C9C003394015002810D306502810DD80281AE72
:100CAC008134C26DC2AF53E67F7591008553948534
:100CBC005495759104854D92854E93D26043E68090
:100CCC00D2AFE52D54066008206A020533020CEC05
:100CDC00306D0D206C0A2065071581158102157485
:100CEC002278003064053065027801E53775F0072D
:100CFC00A4F9E5F028F5F0E9A2F013A2F113A2F2A1
:100D0C0013F537C394785003753778C3E5379538A6
:100D1C004008D266C292C291C290306002A1268570
:100D2C004F92855093D26043E68022207D16C2AF4D
:100D3C00754202C294D295306202D290D2AF759FA6
:100D4C0011020F26C2AF754202C294D293306202D6
:100D5C00D292D2AF759F11020F26307243207D20A4
:100D6C00C2AF75420390013A757B10C290C29330AA
:100D7C006204D291A184D294D2AF759F01020F2646
:100D8C00C2AF75420390013A757B10C292C2953086
:100D9C006204D291A1A4D294D2AF759F21020F26E6
:100DAC00207D17C2AF754203900115C290306202CC
:100DBC00D291D2AF759F01020F26C2AF754203903C
:100DCC000115C292306202D291D2AF759F21020FEF
:100DDC0026207D16C2AF754204C295D293306202B2
:100DEC00D291D2AF759F21020F26C2AF754204C2B9
:100DFC0093D295306202D291D2AF759F01020F2629
:100E0C00307243207D20C2AF754205900129757B5D
:100E1C0020C291C294306204D292C12AD295D2AF30
:100E2C00759F11020F26C2AF75420590014B757B61
:100E3C0008C291C294306204D290C14AD293D2AF0C
:100E4C00759F11020F26207D17C2AF7542059001C8
:100E5C000BC291306202D292D2AF759F11020F2653
:100E6C00C2AF75420590011FC2913062EBD290D295
:100E7C00AF759F11020F26207D16C2AF754206C2B8
:100E8C0093D294306202D292D2AF759F01020F2698
:100E9C00C2AF754206C295D294306202D290D2AFE4
:100EAC00759F21020F26307243207D20C2AF754200
:100EBC000190014B757B08C292C295306204D290AE
:100ECC00C1D0D293D2AF759F21020F26C2AF75420B
:100EDC0001900129757B20C290C293306204D2929A
:100EEC00C1F0D295D2AF759F01020F26207D17C29B
:100EFC00AF75420190011FC292306202D290D2AF04
:100F0C00759F21020F26C2AF75420190010BC29052
:100F1C00306202D292D2AF759F01C2662290010953
:100F2C00757B00C292C291C290C295C294C293C208
:100F3C006222788076090876090876040876FF081C
:100F4C0076030876FF08760B087603087601087698
:100F5C0001788C76010876FF0876FF0876FF087614
:100F6C00FF0876FF0876030876FF0876FF0876FF01
:100F7C000876250876D00876280876500876040876
:100F8C0076FF08760208760008767A0876FF0876EF
:100F9C000108760108760008760308760022788727
:100FAC00E6FFC272BF0302D2727888E6C394036074
:100FBC0008C27DE630E102D27DC27E7889E630E15E
:100FCC0002D27EC3EF94026008758E01D273020FB9
:100FDC00E2758E00C273227880E6149000809378BC
:100FEC00A5F67881E6149000809378A6F67886E6CC
:100FFC001490008D9378A7F67886E6F539C39402A1
:10100C005003753902789CE67538FFB402037538C5
:10101C00A0B4030375388278A3E61490009A93F574
:10102C0066120F2922227896E6FA7897E6FB7888E2
:10103C00E6B40305C3EB940EFB307F047A007BFF10
:10104C00C3EB9AFCC3948250027C827572000572C9
:10105C00EC8572F0A4C3E5F0947D40F222D27F11AE
:0F106C00321205AE7A007B007C101205A4E55C01
:10107B002AFA74003BFBDCF37C04C3EB13FBEA138F
:10108B00FADCF7FEC27F113222E5EF20E603752072
:10109B00000520903FFFE520146006901DFF1460B3
:1010AB00009304600375EF1053D9BF7581C043FFE4
:1010BB008012059F75EF0043B203E5B3240220E7CE
:1010CB000DF521E5E320E0068521B343E301120F83
:1010DB00297580FF75A40075F19075D47F7590000C
:1010EB0075A53F75F23F75D50075A60175E24112E6
:1010FB000F29E4F8F6D8FD756801120F3E1215C5DD
:10110B0078988673753001C2AF1205B81205C812F4
:10111B0005AE1205CF1205AE1205D61205AEC2AF43
:10112B0078FA79FA308707D9FBD8F7021C00120F2F
:10113B00AA120FE31131113278988673120F2975A9
:10114B00881075890275C82475910475D84075A8E7
:10115B002275B80275E690759B80759D0075D10E52
:10116B0075BC5875BB0675BA1175E88012059FD210
:10117B00AF1208BD75360053DACF207E0343DA2059
:10118B00307E0343DA1043DA01C2D8C2711205B8BC
:10119B00D2617B037A0CE55B70077A0CDB030211DF
:1011AB00291205AE207003021129C270E55CC394AD
:1011BB000240E1E52F541F855E5DF55EB55DD5DA26
:1011CB00D5C26153DACF207E0343DA20307E03434E
:1011DB00DA10C2D8C27178A2E67008D274E52F5427
:1011EB00E0F52FC2757529001205B3307409C3E5FC
:1011FB0029940A4002D2751205A478023074027841
:10120B0000C3E55C9840F0C2AF1205C81205C812C6
:10121B0005C8D2AF1205B8754C007888E6B4030246
:10122B0061011205A4788CE6C394015003021301EB
:10123B00E530C394015003021301207435C3E55C00
:10124B0094FF5003021301C2AF1205DDD2AF12059A
:10125B00B3C3E55C940150EFC2AF1205C81205A9E8
:10126B001205C8D2AF1205B3C3E55C94FF40E90287
:10127B00176D7F02D27F11321205B3C2AFC27F113D
:10128B0032AE5CC3E55C947FD2AF407412059FC253
:10129B00AF1205DDD2AFDFDC1169C3EE7897F61222
:1012AB0005B81216071216F07F0AD27F11321205FB
:1012BB00B3C2AFC27F1132AE5CC3E55C947FD2AFD9
:1012CB0050E612059FC2AF1205C81205A91205C838
:1012DB00D2AFDFD61169EE24037896F61205B81259
:1012EB00160712171F1205B31132C3E55C94FF509A
:1012FB0002414502176DC3E55C954C4003855C4C80
:10130B001205B378017988E7B403027805C3E55C6D
:10131B009840024125C2AF1205DD1205DD1205DD35
:10132B00D2AF1205B8753000E4F531F5320531E571
:10133B0031F4703F0532789AE678191460127832DE
:10134B0014600D787D14600878FA14600375320010
:10135B00C3E53298401D120F2912059F15327531C6
:10136B000078998673C2AF1205DDD2AF7898867379
:10137B001205B31205A9E52A7005307402212978EC
:10138B00012074027806C3E55C9840A17888E6C317
:10139B00940360031205B3E52A7003021129C2AF4F
:1013AB00120F29E4F522F523F524F525F526F5672B
:1013BB00D2AF7885E6C333F565E4F544F545F546DC
:1013CB00F547F548F570F52CF52DF5377570087563
:1013DB00BB1012059F1208C1E5E820ECFBA8BDA9C4
:1013EB00BEE97001F888711208C575700875BB10DD
:1013FB00120FAAC2AF7561FF12095D8522618522AA
:10140B0062852263D2AF75220175240175250175A2
:10141B002601856069756A017888E6B40307C27D89
:10142B00307602D27DD268D269753300120E8312E8
:10143B000EB212097D12098412097D120984120958
:10144B007D120BFF1206B8120CED120D3712098428
:10145B00120BEE306E031207142067031208603074
:0E146B0067031208A7120CED120D6612098419
:10147900120BFF306E03120749120CED120DDD122B
:101489000984120BEE306E031207A7120CED120E2F
:101499000C120984120BFF306E03120804120CEDB2
:1014A900120E831209841208C1120BEE120CED12EE
:1014B9000EB21208C51209843069328564618564E7
:1014C90062856069756A0179187A0CC3E5339940B8
:1014D9000FC269D26A8A358564618564630214F62C
:1014E900C3E55C9401400302144C02157C306A1D6B
:1014F900206C1AE535147006C26AD26B814CF53539
:10150900C3E55C9401400302144C02157C75360056
:1015190078FA79A4E760027803C3E55F98505430FC
:101529007404E52A604D7888E6B40317207D052008
:101539007607A14C307602A14C206C07D26C8564E9
:1015490061818B78F0306C058564617820C3E54151
:10155900985002814C306C1BC26CC27D307602D22D
:101569007DD26A753512856461814C0536E55C600A
:1015790002A17F753600C2AF120F297887E6FE7681
:1015890002120FAA7887EEF6E4F522F523F524F581
:1015990025F526F565752C00752D00D2AF1205B31A
:1015A900120F2978A4E66006D292D291D2903074B3
:1015B90009C3E5369404400221296133901A0D7854
:1015C90020121649E520B4550CA3121649E520B49A
:1015D900AA030215E7120F3E121607021606901A01
:1015E9000378807B0A121649A308DBF9901A0F7851
:1015F9008C7B19121649A308DBF9901A2822C2AF6D
:10160900121688121662901A00740E12164EA374DE
:101619000612164EA3741512164E901A0378807B83
:101629000A12164DA308DBF9901A0F788C7B191250
:10163900164DA308DBF912169B121679901A282267
:10164900E493F622E6438F01538FFD75EF0275B7D8
:10165900A575B7F1F0538FFE22438F02438F0175B1
:10166900EF0275B7A575B7F1901A0DF0538FFC22EB
:10167900901A0D7455D14E901A0E74AAD14E227A31
:101689003079D07820901A40D149E520F709A3DABA
:10169900F7227A3079D0901A40E7D14E09A3DAF9C6
:1016A90022AB74A875BB01027980BB02027981BBA8
:1016B90003027982BB04027984BB05027986BB06E1
:1016C900027992BB07027987BB080279A3BB090299
:1016D900799CBB0A027988BB0B027989E8F7227CDD
:1016E900051205B8DCFB22C2AF1205C81205CF12DC
:1016F90005D61205DD1205A91205C81205CF120576
:10170900D61205DD1205A91205C81205CF1205D694
:101719001205DDD2AF22C2AF1205DD1205D61205C0
:10172900CF1205C81205A91205DD1205D61205CF7B
:101739001205C81205A91205DD1205D61205CF1228
:1017490005C8D2AF22AE74AF75C2AF1205C8120573
:10175900C81205C81205A9DEF21205DD1205A9DFB6
:10176900F8D2AF22D1F0D1E8D1E8757401757501CD
:10177900757600F14E7C05AD5C1205B8C3ED955C3C
:1017890070F5C3E55C9401400AC3E55C94FF4032FF
:101799000217A9D1AAD107D1F0C2AF75EF10D1E8CC
:1017A900DCD50576C3E5769403500280C6D1E805F9
:1017B90075E5741490009F93F808C3E57598500275
:1017C90080AED1E8D1E80574C3E574940C50028069
:0D17D9009C120F3ED107C2AF75EF10D1E892
:0319FD0002109441
:101A00000E0615090904FF03FF0B03010155AA0186
:101A1000FFFFFFFFFF03FFFFFF25D0285004FF0259
:091A2000007AFF0101000300FF40
:101A400023585037414661737423202020202020E2
:101A500023424C48454C4923463333302320202031
:101A60002020202020202020202020202020202076
:101C0000C2AFC2D353D9BF7581C043B20343FF8073
:101C1000752438752503B1C975EF0275E24043F1AB
:101C20008053A47F75D4FFD2877DFA780379E67C50
:101C300010752200752300901DD67B0675249875BB
:101C400025013087028142208708D8FBD9F9DCF7CB
:101C500081B4308708D8FBD9F9DCF781B4B189E4C5
:101C600093A3C39A6004DDC381B4DBDBB17B600264
:101C7000812B7B08E493FAA3B15CDBF87A30B15C8A
:101C8000752200752300B17BEAFCEBFDC3ED94FEE9
:101C9000400EB17B8A278B28ED30E0048A828B834B
:101CA000B17B7AC270D8C3ED94FE601350CEBD00F4
:101CB00025EC60097520007521FF0200008100A855
:101CC00027A9280809D804D90281D3B17FEA89AAB3
:101CD000F281C50D81A0C3ED94035049EDA2E092BD
:101CE000007AC5C3E5829400E583941C50902000DF
:101CF00010438F02438F0175B7A575B7F1F030001F
:101D00001FA827A9280809438F01538FFDD804D99C
:101D100002A12089AAE275B7A575B7F1F0A3A10DBC
:101D2000538FFC817C7AC1BD030CE493A3FAB140CC
:101D3000DCF8B138817C817EAA22AB23B15CEBFA5E
:101D4000EA6222752608C3E52313F523E52213F57D
:101D50002250066323A0632201D526EAB1C9B1C986
:101D600075260AEAF4200102D287300102C287B147
:101D7000C9C3134002C201D526EB22B17FEAFB2082
:101D80008702A17F308702A184752608AE24AF2583
:101D9000C3EF13FFEE13FEB1CDB1C9C3EA13308711
:101DA000024480FA30E703632201C3E52313F523DD
:101DB000E52213F52250066323A0632201D526D91C
:101DC000E52265236523F52222AE24AF250E0FDE22
:101DD000FEDFFCD20122424C48656C693437316326
:041DE000F3300601D5
:00000001FF
